:03000000022CDFF0
:0C2CDF0078FFE4F6D8FD758156022D2622
:100EC5000A53746172743A20004950436F6E6E651F
:100ED50063745245510A004950436F6E6E656374E1
:100EE500003E432C562C43432CC0E4E0EFF2E5F0E2
:100EF50020D1E8EDEAEEEC49500A003E432C4D4185
:100F0500432C25303262583A25303262583A253022
:100F15003262583A25303262583A25303262583AB0
:100F250025303262582C4D414320E0E4F0E5F10ACA
:100F3500003E432C5645522C20332E3120EEF22014
:100F450025732025732CC2E5F0F1E8FF20495020D8
:100F5500ECEEE4F3EBFF0A004A616E2032382032F2
:100F65003030380030383A33393A3539003E432C81
:100F75004C442C50524F473A20202020202020203E
:100F8500202020202020202020202020202020205C
:100F9500202020202020202020202020202020204C
:100FA500202020202020202020202020202020203C
:100FB500202020202020202020202020202CC4E0BC
:100FC500F2E020EFF0EEF8E8E2EAE828F4E0E9EBF9
:100FD500290A003E2A2C312CCEF1EDEEE2EDFBE59F
:100FE50020EFE0F0E0ECE5F2F0FB20F1E5F2E5E2E0
:100FF500EEE3EE20E8EDF2E5F0F4E5E9F1E00A00D4
:101005003E412C4130312C2562752E2562752E25E9
:1010150062752E2562752C495020E0E4F0E5F1203B
:10102500E0E4E0EFF2E5F0E00A003E412C41303229
:101035002C2562752E2562752E2562752E25627505
:101045002C495020E0E4F0E5F120EEF1ED2E20F101
:10105500E5F0E2E5F0E00A003E412C4130332C2575
:1010650062752E2562752E2562752E2562752C49B1
:101075005020E0E4F0E5F120F0E5E72E20F1E5F081
:10108500E2E5F0E00A003E412C4130342C25627542
:101095002E2562752E2562752E2562752CCCE0F104
:1010A500EAE020F1E5F2E80A003E412C4130352C1A
:1010B5002562752E2562752E2562752E2562752C85
:1010C500D8EBFEE70A003E532C4130362C256275DD
:1010D5002CC2F0E5ECFF20EEE6E8E42E20EAE2E89B
:1010E500F2E0EDF6E8E820282A3130ECF1290A0093
:1010F5003E2A2C312CC4EEEF2E20EFE0F0E0ECE59B
:10110500F2F0FB20F1E5F2E5E2EEE3EE20E8EDF2A8
:10111500E5F0F4E5E9F1E00A003E422C5330312CCC
:101125002562752CC6E4E0F2FC20E7E0EFF0EEF175
:10113500E020F1EEE5E4E8EDE5EDE8FF20EEF22054
:10114500F1E5F0E2E5F0E00A003E422C5330322CA6
:101155002562752CCEE1ECE5ED20F120F1E5F0E21C
:10116500E5F0EEEC20E1E5E720EAE2E8F2E0EDF675
:10117500E8E90A003E422C5330332C2562752CCF0A
:10118500E5F0E5E7E0EFF3F1EA20EFF0E820EFEE38
:10119500F2E5F0E520F1E2FFE7E820F120F1E5F0E6
:1011A500E2E5F0EEEC0A003E422C5330342C256289
:1011B500752CCDE5F220EFE5F0E5E4E0F7E820E475
:1011C500E8E0E3EDEEF1F2E8EAE820E220F1E5F00F
:1011D500E2E5F00A003E422C5330352C2562752C91
:1011E500CAE0EDE0EB20F8E8F0EEEAEEE2E5F8E043
:1011F500F2E5EBFCEDEEE3EE20EEE1ECE5EDE00AE9
:10120500003E532C5330362C25303262582530326F
:1012150062582530326258253032625825303262A4
:101225005825303262582C4D414320E0E4F0E5F179
:1012350020F8E8F0EEEAEEE2E5F8E0F2E5EBFCEDA9
:10124500EEE3EE20EEE1ECE5EDE00A003E454E442E
:101255000A0044756D705820202020203030203041
:1012650031203032203033203034203035203036B4
:10127500203037203038203039203041203042208E
:1012850030432030442030452030460A003A003AA9
:1012950020000A0044756D70442020202020303045
:1012A500203031203032203033203034203035208A
:1012B500303620303720303820303920304120304A
:1012C500422030432030442030452030460A004536
:1012D5007272206B657900526420656570726F6D5E
:1012E5000A005264204D454D0A00526420436F6444
:1012F500650A0044656275674950204F4E0A0044EF
:10130500656275674950204F46460A004465627517
:101315006755736572204F6E0A004465627567559F
:10132500736572204F46460A0044656275674D73C2
:1013350067204F6E0A0044656275674D7367204FDD
:1013450046460A00436F6E666967206C6F636B21C2
:101355000A00577220656570726F6D0A002053612F
:10136500766520656570726F6D210A004572722081
:101375004D414321004C6F61643E3E002A003C41D3
:1013850030313D003C4130323D003C4130333D0081
:101395003C4130343D003C4130353D003C41303628
:1013A5003D003C21003C5330313D003C5330323D43
:1013B500003C5330333D003C5330343D003C53300A
:0913C500353D003C5330363D007B
:06347D00010B0001090033
:1034E800C2AFC28E438910758BFF758DB7D2ABD230
:0434F8008ED2AF229F
:03001B00022BAC09
:102BAC00C0E0C083C082C0D0C2AFC28E758BFF752F
:102BBC008DB720060675A61E75A6E10509D202E59D
:102BCC000B6002050BE50AD394014002150A050EB1
:102BDC00E50E540F7050D20EE50E543F701AD20011
:102BEC0090668DE0601204F0E0D394B4400A9080BB
:102BFC00007480F0C2AF80FE906688E0600204F042
:102C0C00906104E0600214F090668EE0D394014071
:102C1C0003E014F0300502050CE50DD39464400478
:102C2C00D2068002050DE508D3940140021508D2A6
:0C2C3C008ED2AFD0D0D082D083D0E03256
:1008A400C291C290D2B5C20B7D027C007F07123484
:1008B400608F24E524646060097D017F6012341830
:1008C400D20BE4FDFC7F0B1234608F24E52430E668
:1008D400097D04E4FF12343CD20B7D017C007F07C8
:1008E4001234608F24E5247008FD7FFF123418D27F
:1008F4000B300B03126000C2AFC288C2A8C2AA7533
:100904008900122FFF906341E0B4FA09A3E064CE9A
:1009140070030209A4E4F52474392524F582E4342F
:1009240063F583E4F00524E524B443EC9063417457
:10093400FAF0A374CEF0A374CCF0906347740AF079
:10094400E4A3F0A304F0A3F090634C7403F0A37445
:10095400CCF090633D74FFF0A3F0A3F0E4A3F09017
:1009640063587405F0E4F524E5242401FFE433FE20
:1009740074392524F582E43463F583E0FD1234CF21
:100984000524E524C3944340DFE4F5A775A61E754A
:10099400A6E1907FF0F0A3F09080007480F080FED8
:1009A400D2AF90634C7403F0A374CCF0E490634B27
:1009B400F012280FC2B51232E2C20612323190632D
:1009C40058E0C3940350037403F0D20BC20DC20C5D
:1009D400D293200B077E0E7FC512242EE4906578F7
:1009E400F01234E8C2AFA37408F09062B77424F034
:1009F400E4A3F0906341E09062B9F0906342E09028
:100A040062BAF0906343E09062BBF0906344E0907C
:100A140062BCF0906345E09062BDF0906346E09064
:100A240062BEF0750A01E490657AF0C207C208C29A
:100A340009C20AD2AF75A70775A61E75A6E1200BD9
:100A440018AF24FE7D0312252FE4FF122A627E6371
:100A54007F78E4FB7D0112262990668DE0600374A3
:100A640001F0E4906104F0A37455F0A37481F0E400
:100A7400F50CE4F50D906104E070031233EC90661C
:100A84008EE0B401119080007410F0E490668EF052
:100A9400D20BC20CC20D908008E0F52430E405D2DC
:100AA400077410F0E52430E508D20990800874201A
:100AB400F0E52430E608D2089080087440F0E50C94
:100AC400D394034023908002E4F0908001F090805E
:100AD40000F0E50CD39406400FE4F50CC2039065D6
:100AE4007AF0750A011232319080A0E0700312305E
:100AF4007D9080B8E070031230F79080D0E07003EE
:100B0400123171908000E0701330071012232A9084
:100B14006334EFF0D394004003120026908002E087
:100B24007006908000E06005D205020A76C205E4F2
:100B3400F50C906104E06003020A76300912122178
:100B4400C4906334EFF0D394004005E0FF12001F1B
:100B5400200803020CD512204F906334EFF0700389
:100B6400020A76906378E054BF247F7003020C3845
:100B7400147003020C1024026003020C6B200B0798
:100B84007E0E7FCE12242E300F7920037690635090
:100B9400E07006906354E0605B906684E0FF9063CD
:100BA40050E0B50724906685E0FE906351E0B506F9
:100BB40018906686E0FE906352E0B5060C90668756
:100BC400E0FE906353E06E602B906354E06F7033EB
:100BD400906685E0FF906355E0B50727906686E050
:100BE400FF906356E0B5071B906687E0FF9063575C
:100BF400E0B5070F90657A7401F0120020750A01C0
:100C0400020CD590668474FFF0020CD590668DE0DA
:100C140060037401F090667CE0FF90637AE06F609B
:100C240003020CD590667CE004F0E4F50A90657844
:100C3400F0020CD5300303020CD5906347E0700337
:100C4400020A7612350FD203E4F50A906578F09023
:100C5400668804F0E490667BF0A3F0200B737E0EAC
:100C64007FDC12242E806A90668DE060037401F0AC
:100C7400300352906378E020E74B90637AE0FF9072
:100C8400667BE0FE6F600D906683E07007EE146F84
:100C9400703F801390667BE004F0906334E0FFD3F0
:100CA400940440031228F59060007482F0A3740148
:100CB400F090637AE0906002F07E607F007D031222
:100CC4002F7F020A76300F0920030690668474FF92
:100CD400F0200303020D8AE50A706B122C48EF60C2
:100CE400207E647F78906479E02404FD122F7F9045
:100CF4006683E06003020A76906358E0F50A020A0C
:100D040076906688E0D3943C403C906683E07036ED
:100D140090668804F09062B6E0702B1229ADE490DE
:100D24006478F0A37412F090667CE090647AF0A387
:100D340074FDF090610763A20190647C63A2017F5B
:100D440012121D9D809B1234FCEF6015906000749C
:100D540083F0E4A3F07E607F007D02122F7F020AFD
:100D640076E50A64016003020A76906578E004F08F
:100D7400E0C394055003020CE5C203E490657AF0E5
:100D8400120020020A76E50A64016003020A7690E2
:100D9400657AE014604624FE6042147003020E7803
:100DA40024046003020A76E4F50C200F1390657A9C
:100DB4007404F0906578E05401F0750A01020A7633
:100DC4009080027410F0E490657AF090657804F0F5
:100DD400750AC890668474FFF0020A76906684E00F
:100DE4007003020E679064787480F090647A7401E2
:100DF400F0E4A3F0A304F0A37430F0A3747BF0E454
:100E0400F524747F2524F582E43464F583747DF03D
:100E140074802524F582E43464F583E4F0E5242425
:100E240007906479F07C667D8490634CE0FAA3E0DB
:100E3400FB7F02122E7B7E647F78E5242409FD1259
:100E44002F7F906683E0601B12350FD203E4F50A0E
:100E5400906578F090668804F0E490667BF0A3F0E7
:100E6400020A7690657A7404F0906358E02432F5AF
:100E74000A020A769080027410F0750A039065786D
:100E8400E06401FFF090657A7401F0EF70199063EB
:100E940054E06013FCA3E0FDA3E0FEA3E0FF906632
:100EA40084121B3E020A76906350E0FCA3E0FDA38B
:100EB400E0FEA3E0FF906684121B3E020A7680FEE9
:010EC400220B
:10002600906379E0B444047F0180027F0090637896
:10003600E0B447047E0180027E00EE5F604A906372
:1000460041E090637AF0906342E090637BF09063C6
:1000560043E090637CF0906344E090637DF09063AE
:1000660045E090637EF0906346E090637FF0906396
:10007600797452F09062B063A2019080A863A201E5
:100086007F06121D9D02089A906334E0C3940850BF
:10009600030208A3906341E0FF90637AE06F600378
:1000A6000208A3906342E0FF90637BE06F60030267
:1000B60008A3906343E0FF90637CE06F600302084F
:1000C600A3906344E0FF90637DE06F60030208A3A2
:1000D600906345E0FF90637EE06F60030208A390A3
:1000E6006346E0FF90637FE06F60030208A39063BE
:1000F60079E0B444159062B0E0B4FF0E63A20190BB
:1001060080A863A2017F06121D9D90668DE06003A4
:100116007401F090668E7464F09063797452F09076
:100126006378E0646D60030202A37BFF7A0E79E6D2
:100136001214307BFF7A0F7900906341E0F52DA30E
:10014600E0F52EA3E0F52FA3E0F530A3E0F531A30B
:10015600E0F532121430752DFF752E0F752F5D7573
:1001660030FF75310F7532697BFF7A0F79361214BD
:10017600307BFF7A0F79721214307BFF7A0F79D8B1
:100186001214307BFF7A107905906347E0F52DA3B2
:10019600E0F52EA3E0F52FA3E0F5301214307BFF37
:1001A6007A10792F906350E0F52DA3E0F52EA3E0A9
:1001B600F52FA3E0F5301214307BFF7A10795D90AD
:1001C6006354E0F52DA3E0F52EA3E0F52FA3E0F5AB
:1001D600301214307BFF7A10798B90633DE0F52D59
:1001E600A3E0F52EA3E0F52FA3E0F5301214307B43
:1001F600FF7A1079AE906339E0F52DA3E0F52EA3D2
:10020600E0F52FA3E0F5301214307BFF7A1079CB9E
:10021600906358E0F52D1214307BFF7A1079F512B1
:1002260014307BFF7A11791EA20FE433F52D1214D8
:10023600307BFF7A11794E906683E0F52D121430EB
:100246007BFF7A11797990668DE0F52D1214307B5B
:10025600FF7A1179AC9062B6E0F52D1214307BFF6F
:100266007A1179DAA201E433F52D1214307BFF7A84
:1002760012790690667DE0F52DA3E0F52EA3E0F554
:100286002FA3E0F530A3E0F531A3E0F532121430E8
:1002960012328A7BFF7A12795112143022906378D7
:1002A600E0644C70757E127F5712242E906380E0B6
:1002B600F525A3E0F526E4F5287E127F9212242E7A
:1002C6007D03AF26AE2512252F7E127F9412242E93
:1002D600E4F527852682852583E0FF74822527F5A8
:1002E60082E43463F583EFF00526E52670020525E2
:1002F6000527E527B410DC7E637F82E4FB7D1012C0
:1003060026297E127F9712242E0528E528C39410ED
:1003160040A77E127F9712242E22906378E0646CA9
:10032600705CF5297E127F9912242EE4F528AF29F8
:100336007E007D0312252F7E127F9412242EE4F573
:1003460027A829E6FF74822527F582E43463F5831E
:10035600EFF005290527E527B410E67E637F82E4E2
:10036600FB7D101226297E127F9712242E0528E582
:1003760028C3940840B87E127F9712242E229063D9
:1003860078E0644B7061F527746A2527F582E434BA
:1003960063F583E06032746A2527F582E43463F5F9
:1003A60083E0F46023746A2527F582E43463F583D9
:1003B600E0FF74802527F582E43463F583E0B50712
:1003C600100527E527B408C09061047432F00208CE
:1003D6009A9063787421F0300B0302089A7E127F9C
:1003E600D412242E02089A906378E0B4521A200B95
:1003F600077E127FDC12242E9063787472F07E637F
:100406007F787D08122EFF22906378E0644970455C
:10041600200B077E127FE712242E906380E0F525DD
:10042600A3E0F526E4F527852682852583E0FF747B
:10043600822527F582E43463F583EFF00526E52669
:10044600700205250527E527B480DC7E637F787D6D
:100456008A122EFF22906378E064437079A3E064E9
:10046600527046200B077E127FEF12242E90638077
:10047600E0F525A3E0F526E4F52785268285258384
:10048600E493FF74822527F582E43463F583EFF065
:100496000526E526700205250527E527B480DB7EBF
:1004A600637F787D8A122EFF22906379E06457601D
:1004B600030208A3906380E0F525A3E0F526748285
:1004C6002527F582E43463AD82FC7B80AF26AE251A
:1004D6001233B802089A906378E064446003020518
:1004E6006D906380E0FF6444700302089AEFB431B4
:1004F6000CC20B7E127FF812242E02089A9063809B
:10050600E0B4300CD20B7E137F0412242E02089A1C
:10051600906380E0B4320CD20C7E137F1112242E2D
:1005260002089A906380E0B4330CC20C7E137F1FDE
:1005360012242E02089A906380E0B4340CD20D7E09
:10054600137F2E12242E02089A906380E0B4350C95
:10055600C20D7E137F3B12242E02089A906380E020
:10056600FF12001E02089A906104E07013200B0728
:100576007E137F4912242E9063787421F002089A24
:100586009061047432F0906378E0FFB4510A908071
:10059600007480F0C2AF80FEEF64577045200B07F1
:1005A6007E137F5712242E906381E0906334F0E42B
:1005B600F527906334E0FFE527C39F400302089ABE
:1005C60074822527F582E43463F583E0FF90638027
:1005D600E0252724AFF582E43461F583EFF00527A3
:1005E60080D0906378E06453600302069C200B077A
:1005F6007E137F6212242E906341E0FF9061B8E083
:100606006F703C906342E0FF9061B9E06F7030908C
:100616006343E0FF9061BAE0B50724906344E0FFCE
:100626009061BBE0B50718906345E0FF9061BCE0C0
:10063600B5070C906346E0FF9061BDE06F601690D1
:1006460063787421F0300B0302089A7E137F7112CF
:10065600242E02089AE4F527E4F50DAF27FE74AFC1
:100666002527F582E43461F583E0FD1234CF0527B2
:10067600E527C394FE40E19080007480F0C2AFE4A9
:10068600907FF0F0A3F0907FFD74AAF0A374FFF0C2
:10069600A37455F080FE906378E0644F704C9063CD
:1006A60080E0F525A3E0F526E5264525700A200B12
:1006B600077E137F7A12242E200B077E137F81126A
:1006C600242EE4F52774822527F582E43463F58326
:1006D600E0852682852583F00526E5267002052518
:1006E6000527E527B480DE02089A906378E0FFB418
:1006F60045279080007480F0906380E0FDA3E09031
:100706007FF0CDF0A3EDF0C2AF907FFD74AAF0A309
:1007160074FFF0A37455F080FEEF64656003020871
:100726009A906380E0FFA3E0907FF0CFF0A3EFF014
:10073600E4F525F526D3907FF1E09526907FF0E04D
:1007460095254020E4F50D2526FFE5253401FE8597
:100756002682852583E0FD1234CF0526E526700224
:10076600052580D17E137F83122DF6EF4E60201271
:100776000003906347EFF0120003906348EFF01216
:100786000003906349EFF012000390634AEFF07E96
:10079600137F89122DF6EF4E6020120003906350EE
:1007A600EFF0120003906351EFF0120003906352D2
:1007B600EFF0120003906353EFF07E137F8F122D3C
:1007C600F6EF4E6020120003906354EFF012000320
:1007D600906355EFF0120003906356EFF01200039A
:1007E600906357EFF07E137F95122DF6EF4E602043
:1007F60012000390633DEFF012000390633EEFF0AA
:1008060012000390633FEFF0120003906340EFF095
:100816007E137F9B122DF6EF4E602012000390632D
:1008260039EFF012000390633AEFF0120003906381
:100836003BEFF012000390633CEFF07E137FA112B2
:100846002DF6EF4E60081231D4906358EFF0E4F5C0
:1008560027E4F50DE5272401FFE433FE7439252747
:10086600F582E43463F583E0FD1234CF0527E527EE
:10087600C3944340DC9080007480F0C2AFE4907F64
:10088600F0F0A3F0907FFD74AAF0A374FFF0A374B8
:0D08960055F080FE7E637F787D08122EFFF6
:0108A3002232
:10338000AE07EEC39430400BEED394395005EE24D3
:10339000D0FF22EEC39461400BEED394665005EE4D
:1033A00024A9FF22EEC39441400BEED3944650056E
:0833B000EE24C9FF22AF062242
:1034B5009062AFE004F070069062AEE004F09062B6
:0A34C500AEE0FEA3E0FF12349922EE
:100003001234B5123380EFC454F0FEC0061234B577
:08001300123380D0E02FFF2220
:1031D400E49068B6F01234B59068B7EFF0C3943059
:1031E4004018E0FFD3943950119068B6E02407F5F5
:1031F40082E43461F583EFF080119068B6E024072F
:10320400F582E43461F583E4F0800C9068B6E00460
:10321400F0E0D3940840BE752D00752E00752F0084
:0C322400E4F5307B017A617907121EABE3
:01323000227B
:042DF6008E2A8F2B67
:102DFA009062AEE4F0A374FFF01234B5EF606EF4A3
:102E0A00606B852B82852A83E493B507EC752C01C8
:102E1A00E52B252CF582E4352AF583E49360259089
:102E2A0062AFE0252CFF9062AEE03400FE123499C6
:102E3A00E52B252CF582E4352AF583E493B50704BE
:102E4A00052C80CCE52B252CF582E4352AF583E484
:102E5A009370A6E52C24FFFFE434FFFE9062AFE0F6
:102E6A002FF09062AEE03EF07E007F0122E4FEFF8A
:012E7A002235
:10280F007E137FA7122DF6EF4E70037F01227E13EA
:10281F007FAA122DF6EF4E600C1234B5EF24D024A0
:10282F00FF920F8002D20F7E137FB0122DF6EF4E64
:10283F00600C1234B5EF24D0906683F08005E490DD
:10284F006683F07E137FB6122DF6EF4E600C1234B6
:10285F00B5EF24D090668DF08005E490668DF07E04
:10286F00137FBC122DF6EF4E600C1234B5EF24D04F
:10287F009062B6F08005E49062B6F07E137FC212CC
:10288F002DF6EF4E600C1234B5EF24D024FF9201D9
:10289F008002C20190634163A20190667D63A20131
:1028AF007F06121D9D30013B7E137FC8122DF6EF60
:1028BF004E603012000390667DEFF01200039066B9
:1028CF007EEFF012000390667FEFF0120003906628
:1028DF0080EFF0120003906681EFF0120003906614
:0628EF0082EFF07F0022E1
:10333900906579E0C3947C503D906579E0FE04F096
:1033490074B72EF582E43462F583EFF0BF0A279053
:103359006579E0FF04F074B72FF582E43462F583F0
:10336900E4F0906579E0FF122B0C9065797408F010
:073379009062B8E004F022AD
:103231009080007480F090633963A201F583F58278
:1032410063A2017F08121D9D90634163A2019080DA
:103251008863A2017F0A121D9D908092E4F0A374FD
:1032610032F0A37401F090634BE0FF9080B1F090D5
:1032710080E1EFF09080957455F0A3F09080007498
:0932810001F090800974F0F022C4
:10307D00908009E04410F09080A0E0706C9080A1E9
:10308D007482F09080A874FFF0A3F0A3F0A3F07FFA
:10309D00039080AEEFF07FCBA3EFF07F039080AC79
:1030AD00EFF0A374CBF09080007402F09068AA1238
:1030BD001B4A000000009068AAE0908040F09068E4
:1030CD00ABE0908041F09068ACE0908042F0906869
:1030DD00ADE0908043F0A3E4F0A3F0A3F0A3F09053
:0930ED008018F0A3F0A3F0A3F099
:0130F60022B7
:10317100908009E04440F09080D17482F090634CDB
:10318100E0FF9080DEF090634DE0FF9080DFF090F3
:1031910080027402F09068AE121B4A000000009099
:1031A10068AEE0908058F09068AFE0908059F09060
:1031B10068B0E090805AF09068B1E090805BF0A335
:1031C100E4F0A3F0A3F0A3F0908030F0A3F0A3F01B
:0231D100A3F069
:0131D30022D9
:1030F700908009E04420F09080B8E0706C9080B92F
:103107007482F07F039080C6EFF07FCDA3EFF07F4E
:10311700039080C4EFF0A374CDF09080C074FFF0EB
:10312700A3F0A3F0A3F09080017402F09068B212AC
:103137001B4A000000009068B2E090804CF0906855
:10314700B3E090804DF09068B4E090804EF09068C6
:10315700B5E090804FF0A3E4F0A3F0A3F0A3F090C4
:093167008024F0A3F0A3F0A3F012
:01317000223C
:102E7B008C258D26A907EAFDE975F018A424ACFF73
:102E8B00E5F034808F82F583EDF0EBFDE975F018FA
:102E9B00A4FFAEF024ACFBEE34808B82F583A3ED64
:102EAB00F08526828C83E0FDEF24A8FFEE3480FEB4
:102EBB008F82F583EDF08526828C83A3E08F828E43
:102ECB0083A3F0852682852583A3A3E0FDE975F016
:102EDB0018A424A8FFE5F03480FE8F82F583A3A30A
:102EEB00EDF08526828C83A3A3A3E08F828E83A330
:042EFB00A3A3F0227B
:062EFF008D2AAB07AA06B4
:102F0500908000E020E5729068AAE0FCA3E0FDA3B4
:102F1500E0FEA3E0F52E8E2D8D2C8C2BAE02AF039B
:102F25008E838F8263A201E52D540744C0F5838506
:102F35002E8263A201AF2A121E0FE4FCFDFEE52ED0
:102F4500252AF52EEE352DF52DED352CF52CEC3508
:102F55002BF52B908040E52BF0A3E52CF0A3E52D78
:102F6500F0A3E52EF09080007420F0AF2EAE2DADCD
:092F75002CAC2B9068AA121B3E43
:012F7E002230
:062F7F008D25AB07AA0638
:102F8500908002E020E5729068AEE0FCA3E0FDA32E
:102F9500E0FEA3E0F5298E288D278C26AE02AF032F
:102FA5008E838F8263A201E528540744D0F583857B
:102FB500298263A201AF25121E0FE4FCFDFEE5295F
:102FC5002525F529EE3528F528ED3527F527EC35A6
:102FD50026F526908058E526F0A3E527F0A3E528F9
:102FE500F0A3E529F09080027420F0AF29AE28AD5A
:092FF50027AC269068AE121B3EC9
:012FFE0022B0
:022A62008F25BE
:102A6400908001E030E5037F00229068B2E0FCA38F
:102A7400E0FDA3E0FEA3E0F5298E288D278C2690A7
:102A8400667D63A201E528540744C8F5838529823D
:102A940063A2017F06121E25E5292406F529E435E3
:102AA40028F528E43527F527E43526F52690657BB7
:102AB40063A201E528540744C8F58385298263A2EB
:102AC40001AF25121E25E4FCFDFEE5292525F52987
:102AD400EE3528F528ED3527F527EC3526F5269033
:102AE400804CE526F0A3E527F0A3E528F0A3E5292B
:102AF400F09080017420F0AF29AE28AD27AC269069
:072B040068B2121B3EAF2571
:012B0B0022A7
:10232A009081E0E0F52505250525052505250525E6
:10233A0005250525052505250525908010E0F528A4
:10234A00A3E0F529A3E0F52AA3E0F52B9081E1E0CB
:10235A00F525052505250525052505250525052533
:10236A00052505250525908014E0F52CA3E0F52D1B
:10237A00A3E0F52EA3E0F52FE52EB52A08E52FB543
:10238A002B037F0022E4F525E52E540744E0F5836C
:10239A00852F8263A20190637863A2017F08121ECF
:1023AA005590637A63A2019062B063A2017F06121C
:1023BA001D9D906378E0F526A3E0F527E4F52590C6
:1023CA006378E0702AA3E024F8F525E52E54074443
:1023DA00E0F583852F8274082582F582E43583F53A
:1023EA008363A20190637863A201AF25121E55AEE2
:1023FA0026E4FCFDE52F2527F52FE52E3EF52EEDEB
:10240A00352DF52DEC352CF52C908014E52CF0A308
:10241A00E52DF0A3E52EF0A3E52FF090800074409F
:03242A00F0AF25EB
:01242D00228C
:10204F009081E6E0F52505250525052505250525BE
:10205F0005250525052505250525908028E0F5286A
:10206F00A3E0F529A3E0F52AA3E0F52B9081E7E0A3
:10207F00F525052505250525052505250525052511
:10208F0005250525052590802CE0F52CA3E0F52DE1
:10209F00A3E0F52EA3E0F52FE4F525E52EB52A0AEA
:1020AF00E52FB52B05C2080221A9E52E540744F0F0
:1020BF00F583852F8263A20190637863A2017F0865
:1020CF00121E55906378E0F526A3E0F527E5274526
:1020DF002670099080027410F07F0022906684E0D1
:1020EF00FFF4602D90637AE06F7076906685E0FF65
:1020FF0090637BE06F706A906686E0FF90637CE090
:10210F006F705E906687E0FF90637DE06F60228066
:10211F005090637AE0906684F090637BE0906685E0
:10212F00F090637CE0906686F090637DE090668728
:10213F00F0906378E0702AA3E024F8F525E52E549B
:10214F000744F0F583852F8274082582F582E435E4
:10215F0083F58363A20190637863A201AF25121EFA
:10216F0055AE26E4FCFDE52F2527F52FE52E3EF590
:10217F002EED352DF52DEC352CF52CAF2BAE2AADE4
:10218F0029AC28AB2FAA2EA92DA82CD3121B2D407A
:10219F00099080027410F07F002290802CE52CF0C3
:1021AF00A3E52DF0A3E52EF0A3E52FF090800274A8
:0421BF0040F0AF2518
:0121C30022F9
:1021C4009081E3E0F525052505250525052505254B
:1021D4000525052505250525052590801CE0F52800
:1021E400A3E0F529A3E0F52AA3E0F52B9081E4E030
:1021F400F52505250525052505250525052505259B
:10220400052505250525908020E0F52CA3E0F52D76
:10221400A3E0F52EA3E0F52FE4F525E52EB52A0A73
:10222400E52FB52B05C20902230FE52E540744E818
:10223400F583852F8263A20190600463A2017F0E5F
:10224400121E6B906004E0F526A3E0F52790600C65
:10225400E0FFF4604590667DE0FEEF6E706EA3E0F3
:10226400FF90600DE06F706490667FE0FF90600EF9
:10227400E06F7058906680E0FF90600FE06F704CE4
:10228400906681E0FF906010E06F7040906682E09D
:10229400FF906011E06F60048032D2D9906004E056
:1022A400702AA3E024F2F525E52E540744E8F583CB
:1022B400852F82740E2582F582E43583F58363A22B
:1022C4000190600463A201AF25121E6BAE26E4FCEC
:1022D400FDE52F2527F52FE52E3EF52EED352DF5C1
:1022E4002DEC352CF52CAF2BAE2AAD29AC28AB2F19
:1022F400AA2EA92DA82CD3121B2D5006E52745265E
:1023040070099080017410F07F0022908020E52CE9
:10231400F0A3E52DF0A3E52EF0A3E52FF0908001C6
:052324007440F0AF253C
:012329002291
:04242E008E2A8F2B38
:10243200E4F52CF52D908000E030E511052DE52D19
:102442007002052CD394E8E52C940340E8908000B8
:10245200E030E50302252E9068AAE0FCA3E0FDA38C
:10246200E0FEA3E0F5318E308D2F8C2EE531FFE5B5
:10247200305407FEE42FF52DEE34C0F52C852D8265
:10248200F5837423F0052DE52D7002052C532CC71E
:10249200F582852C83740AF0052DE52D7002052C3A
:1024A200532CC790634163A201852C83852D8263DF
:1024B200A2017F06121E0F7406252DF52DE4352C80
:1024C200F52C852A83852B8263A201852C83852D99
:1024D2008263A201121DF3E4FCFDFE9068AAE0F8FB
:1024E200A3E0F9A3E0FAA3E02FFFEE3AFEED39FDF7
:1024F200EC38FCEF2408FFE43EFEE43DFDE43CFC46
:102502009068AA121B3E9068AAE0908040F0906802
:10251200ABE0908041F09068ACE0908042F090682F
:0C252200ADE0908043F09080007420F049
:01252E00228A
:062629008E2A8F2B8D2C80
:10262F00E4F52DF52E908000E030E511052EE52E16
:10263F007002052DD394E8E52D940340E8908000B7
:10264F00E030E50302271C9068AAE0FCA3E0FDA39D
:10265F00E0FEA3E0F5328E318D308C2FE532FFE5B1
:10266F00315407FEE42FF52EEE34C0F52D852E8262
:10267F00F5837423F0052EE52E7002052D532DC71B
:10268F00F582852D83EBF0052EE52E7002052D5377
:10269F002DC790634163A201852D83852E8263A28E
:1026AF00017F06121E0F7406252EF52EE4352DF52B
:1026BF002D852A83852B8263A201852D83852E820A
:1026CF0063A201AF2C121E0F7408252CF52CFFE40A
:1026DF00FCFDFEE5322FF532EE3531F531ED3530BB
:1026EF00F530EC352FF52F908040E52FF0A3E53036
:1026FF00F0A3E531F0A3E532F09080007420F0AF45
:0D270F0032AE31AD30AC2F9068AA121B3EE7
:01271C00229A
:022B0C008F3EFA
:102B0E00E4F53FF540908000E030E5110540E540EA
:102B1E007002053FD394E8E53F940340E8908000AF
:102B2E00E020E5799068AAE0FCA3E0FDA3E0FEA317
:102B3E00E0F5448E438D428C41E544FFE543540756
:102B4E00FEE42FF540EE34C0F53F9062B763A2016C
:102B5E00853F8385408263A201AF3E121E0FE4FCC7
:102B6E00FDFEE544253EF544EE3543F543ED354295
:102B7E00F542EC3541F541908040E541F0A3E54248
:102B8E00F0A3E543F0A3E544F09080007420F0AF8D
:0D2B9E0044AE43AD42AC419068AA121B3E0C
:012BAB002207
:06252F008E2A8F2BAB0584
:10253500E4F52CF52D908000E030E511052DE52D15
:102545007002052CD394E8E52C940340E8908000B4
:10255500E030E5030226289068AAE0FCA3E0FDA38D
:10256500E0FEA3E0F5318E308D2F8C2EE531FFE5B1
:10257500305407FEE42FF52DEE34C0F52C852D8261
:10258500F5837423F0052DE52D7002052C532CC71A
:10259500F582852C83EBF0052DE52D7002052C9039
:1025A500634163A201852C83852D8263A2017F0689
:1025B500121E0F7406252DF52DE4352CF52C532C04
:1025C500C7E52A852D82852C83F0052DE52D700222
:1025D500052C532CC7F582852C83E52BF0052DE5BD
:1025E5002D7002052C532CC7E531240AF531E4354D
:1025F50030F530E4352FF52FE4352EF52E9080405B
:10260500E52EF0A3E52FF0A3E530F0A3E531F0903A
:1026150080007420F0AF31AE30AD2FAC2E9068AA9B
:03262500121B3E47
:01262800228F
:10349900E5D220E0FBC2AF438E2075D2028F828E27
:0B34A90083E0FFE4F5D2538EDFD2AFCA
:0134B40022F5
:1034CF00E5D220E0FBC2AF43D2028F828E83EDF0B4
:0934DF0075D25063D250D2AF2225
:102FFF00E4FDED2401FFE433FE12349974392DF50D
:10300F0082E43463F583EFF00DBD3FE6E4FDED247C
:10301F007FFFE433FE123499742F2DF582E434616F
:10302F00F583EFF0742F2DF582E43461F583E070B2
:10303F001B742F2DF582E43461F5837420F0743006
:10304F002DF582E43461F583E4F080040DBD80BE7C
:10305F00E49061AEF0FDEDFF7E0012349974AF2D58
:0D306F00F582E43461F583EFF00DBDFEE95C
:01307C002231
:0233B8008B2A5E
:1033BA00A2AF9210C2AF85A22B53A2FE8E838F8238
:1033CA0005A28C838D827409121E99E52A53A2FEE6
:1033DA0043A220121E9B53A2DF852BA2A21092AFFA
:0133EA00FFE3
:0133EB0022BF
:10346000A2AF9210C2AF8C838D82EF121E9943A23D
:0C34700020121E9B53A2DFA21092AFFF9F
:01347C00222D
:023418008F25FE
:10341A00A2AF9210C2AFE4F5838D827406121E9990
:10342A00E52543A220121E9B53A2DFA21092AF7F72
:01343A000190
:01343B00226E
:02343C008F25DA
:10343E00A2AF9210C2AFE4F5838D82740A121E9968
:10344E00E52543A220121E9B53A2DFA21092AF7F4E
:01345E00016C
:01345F00224A
:101CC200A907E7FFA805EF93C3966008403B74FCA1
:101CD2002FFF80F00F08EF93C3966008402B74FB30
:101CE2002FFF80E00F08EF93C3966008401B74FA41
:101CF2002FFF80D00F08EF93D3966008400B74F942
:101D02002FFF80C01F1F1F1F1FEF54FEF80303F792
:101D1200E893FC08E893FD08E893FE08E893FF22A5
:101D220009E993C39D6008402974FB29F980F109F0
:101D3200E993C39E6008401A74FA29F980E209E91E
:101D420093D39F6008400B74F929F980D3191919AC
:101D52001919E9C313C313FF22740093F8ECC39853
:101D62004024701F740193F8EDC3984019701474E5
:0E1D72000293F8EEC398400E7009740393F8C4
:101D8000EFC39840037F00227F0122EDF8E6F008C0
:101D9000A3DFFA22EDF8E0F608A3DFFA22E0A3635E
:101DA000A201F0A363A201DFF475A2002263A201E5
:101DB000F0A363A20122E0A363A201F0A363A20146
:101DC000E0A363A201F0A363A201E463A201F0A374
:101DD00063A201DFE175A20022E0A363A2016DFE10
:101DE000936CFDEE058393FC158363A201DFEA7516
:101DF000A200227F00E493A363A201F00F600CA372
:101E0000E583C2E3F58363A20180EA75A20022E0C4
:101E1000A363A201F0A3E583C2E3F58363A201DF1C
:101E2000EE75A20022E0A363A201F0A3E583C2E461
:101E3000D2E3F58363A201DFEC75A20022E0A36385
:101E4000A201F0A3E58344F8C2E5F58363A201DFB4
:101E5000EC75A20022E583C2E3F583E0A363A2014F
:101E6000F0A363A201DFEE75A20022E583C2E4D2F3
:0A1E7000E3F583E0A363A201F0A3F1
:101E7A0063A201DFEC75A20022E58344F8F583E052
:101E8A00A363A201F0A363A201DFEE75A20022F907
:101E9A0022C002C004C00612FFF0D006D004D0024D
:011EAA002215
:10172A003E2A2C312CCFE0F0E0ECE5F2F0FB20E091
:10173A00F1E8EDF5F0EEEDEDEEE3EE20EFEEF0F28E
:10174A00E00A003E4C2C4930312C256C752CD1EA2C
:10175A00EEF0EEF1F2FC20EEE1ECE5EDE02C3530B6
:10176A002C3130302C3330302C3630302C31323072
:10177A00302C323430302C343830302C393630304A
:10178A002C31393230302C33383430302C3537362E
:10179A0030302C3131353230300A003E422C49305B
:1017AA00322C2562752CC2FBF1F2E0E2EBFFF2FC6F
:1017BA002052545320EFF0E820EFE5F0E5E4E0F79B
:1017CA00E50A003E532C4930332C2562752CC7E0BC
:1017DA00E4E5F0E6EAE020F1F2E0F0F2E020EFE5FD
:1017EA00F0E5E4E0F7E8282A3130ECF1290A003C78
:1017FA0021003C4930313D003C4930323D003C49F2
:10180A0030333D003C4930343D003C4930353D00E1
:10181A003C4930363D003C4930373D003C49303880
:10182A003D000AC1F3F4E5F020E7E0EDFFF2210004
:10183A000A4F55543E000A3C0020212121435243BD
:10184A00204552523A20000089129B24AD36BF48E7
:10185A00C15AD36CE57EF78108931AA52CB73EC905
:10186A0040DB52ED64FF76028B109926AF34BD4AF5
:10187A00C358D16EE77CF5830A9118A72EB53CCBE5
:10188A0042D950EF66FD74048D169F20A932BB4CD5
:10189A00C55ED768E17AF3850C971EA128B33ACDC5
:1018AA0044DF56E960FB72068F149D22AB30B94EB5
:1018BA00C75CD56AE378F1870E951CA32AB138CFA5
:1018CA0046DD54EB62F97008811A932CA53EB740A5
:1018DA00C952DB64ED76FF89009B12AD24BF36C185
:1018EA0048D35AE56CF77E0A8318912EA73CB54275
:1018FA00CB50D966EF74FD8B029910AF26BD34C365
:10190A004AD158E76EF57C0C851E9728A13AB34454
:10191A00CD56DF60E972FB8D049F16A920BB32C544
:10192A004CD75EE168F37A0E871C952AA338B14634
:10193A00CF54DD62EB70F98F069D14AB22B930C724
:10194A004ED55CE36AF17800112332465765748CF0
:10195A009DAFBECADBE9F810013322564775649C75
:10196A008DBFAEDACBF9E82130021367764455AD64
:10197A00BC8E9FEBFAC8D93120120377665445BD55
:10198A00AC9E8FFBEAD8C94253617004152736CE44
:10199A00DFEDFC8899ABBA5243716014053726DE35
:1019AA00CFFDEC9889BBAA6372405125340617EF24
:1019BA00FECCDDA9B88A9B7362504135241607FF15
:1019CA00EEDCCDB9A89A8B8495A7B6C2D3E1F0080C
:1019DA00192B3A4E5F6D7C9485B7A6D2C3F1E018F5
:1019EA00093B2A5E4F7D6CA5B48697E3F2C0D129E4
:1019FA00380A1B6F7E4C5DB5A49687F3E2D0C139D5
:101A0A00281A0B7F6E5C4DC6D7E5F48091A3B24AC3
:101A1A005B69780C1D2F3ED6C7F5E49081B3A25AB4
:101A2A004B79681C0D3F2EE7F6C4D5A1B082936BA3
:101A3A007A48592D3C0E1FF7E6D4C5B1A092837B94
:071A4A006A58493D2C1E0FF4
:1034830052668F00000000000000000000000000F2
:05349300000000000034
:01001E0022BF
:03002300022D6B40
:0B2D6B00C0E0C083C082C0D075D0184B
:102D760030984BC298750B01AF99E545700EEF641C
:102D860055703BF54C754501D2918032E555702E54
:102D960074A1254CF582E43466F583EFF0E54CB476
:102DA6000104EF04F546E54C600AB5460F04F555F7
:102DB600C2918008EF64556003754500054C309953
:102DC60026301A21D290E553B54B0AC21AD21CC23C
:102DD60090D296801074A12553F582E43467F5836A
:072DE600E0F5990553C299C5
:092DED00D0D0D082D083D0E032B6
:10328A007BFF7A17792A1214309068A4E0FEA3E033
:10329A00FFC3E49FFFE49EFEAB07FA3395E0F9F81B
:1032AA007F007E8C7D0A7C00121A8D8F308E2F8DC6
:1032BA002E8C2D7BFF7A17794D1214307BFF7A17EB
:1032CA0079A5A21BE433F52D1214307BFF7A177906
:0832DA00CD85482D12143022AD
:10271D007E177FF9122DF6EF4E70037F01227E1783
:10272D007FFC122DF6EF4E60231231D4A804A905BB
:10273D00AA06AB077F007E8C7D0A7C00121A8D12D3
:10274D001B1F9068A4EEF0A3EFF0800A9068A474AC
:10275D00FFF0A374B8F07E187F02122DF6EF4E60D5
:10276D000C1234B5EF24D024FF921B8002C21B7EC5
:10277D00187F08122DF6EF4E60071231D48F488066
:10278D0003E4F5487E187F0E122DF6EF4E6007120A
:10279D0031D48F478003E4F5477E187F14122DF650
:1027AD00EF4E60071231D48F568003E4F5567E1834
:1027BD007F1A122DF6EF4E600A1231D49068A1EFF8
:1027CD00F080069068A17401F07E187F20122DF61E
:1027DD00EF4E600A1231D49068A2EFF08006906837
:1027ED00A27402F07E187F26122DF6EF4E600A12AB
:1027FD0031D49068A3EFF080069068A37403F07F46
:02280D000022A7
:1032E200C21AC21CE4F545F553F54BF54CF50BC279
:1032F2001975540912271DD296C2ADE4F5C9D2CD73
:10330200D2CCC2C9C2CAF5CDF5CC9068A4E0F5CB47
:10331200A3E0F5CA85CBCD85CACCE4F598D29E430D
:103322008740C29FC2ACC298C29975B81075B710D7
:07333200D2CAD29CD2AC22EA
:01001F0022BE
:1029AD00E4FF0F2407F582E43461F583E554F00F5D
:1029BD0074072401F582E43461F583E4F07C667DCF
:1029CD0094FEED1DAA0470011CF5828A83E0FBAA1A
:1029DD00070F74072AF582E43461F583EBF00EBE20
:1029ED0004E07C667D98E4FEED1DAA0470011CF5E3
:1029FD00828A83E0FBAA070F74072AF582E434610B
:102A0D00F583EBF00EBE04E07C667D9CE4FEED1DCF
:102A1D00AA0470011CF5828A83E0FBAA070F7407D4
:102A2D002AF582E43461F583EBF00EBE04E07C669A
:102A3D007DA0E4FEED1DAA0470011CF5828A83E0E1
:102A4D00FBAA070F74072AF582E43461F583EBF0D6
:042A5D000EBE04E0C5
:012A61002252
:08350700C2992099FDD299221E
:07350F00D2CAD29CD2AC220B
:1028F5008F25301A0E300B030229AC7E187F2C125F
:10290500242E2290637BE0F5547F7C7583630582DA
:1029150063A2019067A463A201E52524FCFF121DB3
:102925009D9067A17455F0A3F0E52524FEA3F0E57D
:102935002504F54BE4F54FF550E52524FCF5527FCC
:10294500A4758367058263A20190185163A201AF44
:1029550052AE51AD50AC4F121DD98F528E518D5084
:102965008C4F749F254BF582E43467F583E550F071
:1029750074A0254BF582E43467F583E54FF0E4F563
:1029850053D21AC296E5486004F50880031235074C
:10299500200B127E187F3A12242E7E677FA1E4FB5E
:0829A500AD4B122629C21C22D1
:102C4800E5557002FF22E55524FEF5259066A3633D
:102C5800A20190647C63A201AF25121D9DE4F54595
:102C6800F555906478F0E52524FEA3F090667CE0A5
:102C780090647AF0A37419F0E4F54FF55085255265
:102C88007F7C758364058263A20190185163A20159
:102C9800AF52AE51AD50AC4F121DD98F528E518DDF
:102CA800508C4F200B127E187F4012242E7E647F9A
:102CB8007CE4FBAD25122629E550454F6016200B14
:102CC800107E187F4312242E7D03AF50AE4F12257D
:062CD8002F7F00227F01A6
:012CDE0022D3
:0100200022BD
:1033EC00300004C2000549300E04C20E054DE5083C
:1033FC00B40106E4F508123507301A0CE549D394EC
:0C340C00144008C21AD21C22E4F5492228
:0B34FC00301C05C21C7F01227F002253
:102CEB000208A4E493A3F8E493A34003F68001F253
:102CFB0008DFF48029E493A3F85407240CC8C333EA
:102D0B00C4540F4420C8834004F456800146F6DFB8
:102D1B00E4800B010204081020408090347DE47E97
:102D2B00019360BCA3FF543F30E509541FFEE493AD
:102D3B00A360010ECF54C025E060A840B8E493A374
:102D4B00FAE493A3F8E493A3C8C582C8CAC583CA9F
:102D5B00F0A3C8C582C8CAC583CADFE9DEE780BE57
:013498000033
:101A510075F008758200EF2FFFEE33FECD33CDCC4C
:101A610033CCC58233C5829BED9AEC99E5829840CF
:101A71000CF582EE9BFEED9AFDEC99FC0FD5F0D6AC
:101A8100E4CEFBE4CDFAE4CCF9A88222B800C1B9D6
:101A91000059BA002DEC8BF084CFCECDFCE5F0CB14
:101AA100F97818EF2FFFEE33FEED33FDEC33FCEB4D
:101AB10033FB10D703994004EB99FB0FD8E5E4F908
:101AC100FA227818EF2FFFEE33FEED33FDEC33FCF5
:101AD100C933C910D7059BE99A4007EC9BFCE99AE9
:101AE100F90FD8E0E4C9FAE4CCFB2275F010EF2F2E
:101AF100FFEE33FEED33FDCC33CCC833C810D7072E
:101B01009BEC9AE899400AED9BFDEC9AFCE899F868
:0E1B11000FD5F0DAE4CDFBE4CCFAE4C8F922FB
:0E1B1F00C3E49FFFE49EFEE49DFDE49CFC22D7
:101B2D00EB9FF5F0EA9E42F0E99D42F0E89C45F00E
:011B3D002285
:0C1B3E00ECF0A3EDF0A3EEF0A3EFF0221A
:101B4A00A8828583F0D083D082121B61121B611296
:101B5A001B61121B61E473E493A3C583C5F0C583BB
:101B6A00C8C582C8F0A3C583C5F0C583C8C582C8E5
:011B7A002248
:1013CE00E539242DF8E6053922782A301702782DD2
:1013DE00E475F001121C22021B7B2010EB7F2ED233
:1013EE00108018EF540F2490D43440D4FF30140BD7
:1013FE00EF24BFB41A0050032461FFE53A600215D2
:10140E003A053DE53D7002053C30170D782AE4752E
:10141E00F001121C22EF021BC10233397403D217E2
:10142E008003E4C217F5398B2A8A2B892CE4F53A0E
:10143E00F53CF53DE53A60077F2012140980F575FD
:10144E003BFFC211C210C212C213C215C216C2187D
:10145E001213D7FF700D3017057F0012141AAF3D0F
:10146E00AE3C22B4255FC2D5C2141213D7FF24D0CE
:10147E00B40A00501A75F00A783A30D50508B6FF4E
:10148E000106C6A426F620D5047002D21380D924F4
:10149E00CFB41A00EF5004C2E5D21402161AD211BC
:1014AE0080C6D21080C0D21280BCD2D580BAD215DE
:1014BE0080B47F201214092012077401B53A00403F
:1014CE00F11213CEFF121409021442D218D2168052
:1014DE00951213CEFB1213CEFA1213CEF94A4B709D
:1014EE000679EB7A167BFF20122EE53A602A7E00F3
:1014FE008E82758300121B9460060EEE653B70F0B3
:10150E00C2D5EBC0E0EAC0E0E9C0E0EE121661D051
:10151E00E0F9D0E0FAD0E0FB121B7BFF60AAEBC033
:10152E00E0EAC0E0E9C0E0121409D0E02401F9D0ED
:10153E00E03400FAD0E0FBE53B0460DCD53BD9801B
:10154E00877BFF7A16795DD212809C7910800279A2
:10155E0008C216C2188008D2D5790A8004790AC248
:10156E00D5E53B047002F53BE4FAFDFEFF1213CE07
:10157E00FC7B082011131213CEFD7B1030100A12C3
:10158E0013CEFE1213CEFF7B20EC3382D592D550B4
:10159E0013C3E43010069FFFE49EFEE42011039D6A
:1015AE00FDE49CFCE4CBF8C211EC700CCFCECDCC9C
:1015BE00E824F8F870F38017C3EF33FFEE33FEED37
:1015CE0033FDEC33FCEB33FB994002FB0FD8E9EB18
:1015DE00301105F8D0E0C448B211C0E00AEC4D4E0F
:1015EE004F78207B0070C2EAB53B0040BCC0E012D1
:1015FE001663D0F0D0E0201104C4C0E0C4B211C014
:10160E00F01213F2D0F0D5F0EB021442121C81143A
:10161E00DF5315595814B04C14AC42155D4F156577
:0F162E004415654914C543156B55154F46154FA7
:10163D0045154F47170B5014B42D14B82E14DB2B32
:10164D0014BC2314D92016F42A147448000014D3A2
:10165D003F3F3F00790AA2D5201314301509B91068
:10166D00020404B9080104A2D52016025001042079
:10167D0012689212B53A005034C0E07F2030131931
:10168D007F30A21272167215500F1216BAC212C204
:10169D0016C215C2187F30800F301503E9C0E01255
:1016AD001409301503D0E0F9D0E0B53ACC30151758
:1016BD007F30B9100C1214097F583014077F7880D1
:1016CD0003B908031214093012057F2D0214097F86
:1016DD00202018F87F2B2016F322921280CF286E2F
:1016ED00756C6C2900D2111213CE3011F8C211781D
:1016FD003A30D50108F60214742D5043495812138F
:10170D00CE2403B405004001E4901706931213FA9A
:0D171D00743A1213FAD213753A04021559EA
:101EAB008B2A8A2B892CE4F536F535F534F533F589
:101EBB0031F532E52E452F452D6012EBC0E0EAC01F
:101ECB00E0E9C0E0AB2DAA2EA92F121C32AB2A05DC
:101EDB002CE52CAA2B7002052B14F9121B7BF53762
:101EEB00C394094007E537D3940D40E1E5376420EF
:101EFB0060DBE537B42D054332038016E537B42B91
:101F0B0005433201800C74FF252CF52C74FF352B07
:101F1B00F52BE53060046410703FAB2AAA2BA92C7B
:101F2B00121B7B64306009E530702E75300A8029F6
:101F3B00900001121B94FF64786004EFB4581343B4
:101F4B0032017530107402252CF52CE4352BF52B52
:101F5B008007E5307003753008AB2A052CE52CAAF9
:101F6B002B7002052B14F9121B7BF537C3946140C0
:101F7B000AE537D3947A50035337DF74D02537F5FE
:101F8B0037C3940A400CE5379411406D74F925372B
:101F9B00F537E537D39530506043320185363B85B5
:101FAB00353A853439853338AF307E00E4FCFDABF0
:101FBB0036AA35A934A833121BD3C8ECC8C9EDC94E
:101FCB00CAEECACBEFCBE4FCFDFEEB2537F536EEC4
:101FDB003AF535ED39F534EC38F533AF36AE35AD82
:101FEB0034FCAB3BAA3AA939A838D3121B2D5003AA
:101FFB00021F64433204021F64E53220E003E480D5
:10200B002DE52E452F452D601EAB2AE52C24FFF91F
:10201B00E52B34FFFAEBC0E0EAC0E0E9C0E0AB2D02
:10202B00AA2EA92F121C32E53230E20774FFFFFEF5
:10203B00FDFC22E532AF36AE35AD34AC3330E103C7
:04204B00021B1F2233
:101B7B00BB010689828A83E0225002E722BBFE0268
:091B8B00E32289828A83E493229B
:101B9400BB010CE58229F582E5833AF583E0225006
:101BA40006E92582F8E622BBFE06E92582F8E22250
:0D1BB400E58229F582E5833AF583E493226A
:101BC100BB010689828A83F0225002F722BBFE0103
:021BD100F322FD
:101BD300E88FF0A4CC8BF0A42CFCE98EF0A42CFCB1
:101BE3008AF0EDA42CFCEA8EF0A4CDA8F08BF0A42F
:101BF3002DCC3825F0FDE98FF0A42CCD35F0FCEB8E
:101C03008EF0A4FEA9F0EB8FF0A4CFC5F02ECD3952
:0F1C1300FEE43CFCEAA42DCE35F0FDE43CFC22BF
:101C2200FAE6FB0808E6F925F0F618E6CA3AF622C3
:101C3200BB011A89828A83D0F0D0E0F8D0E0F9D0D3
:101C4200E0FAD0E0FBE8C0E0C0F0021CB05016E9B8
:101C5200F8D083D082D0E0F9D0E0FAD0E0FBC082A5
:101C6200C083021CA7BBFE16E9F8D083D082D0E065
:0F1C7200F9D0E0FAD0E0FBC082C083021CB92297
:101C8100D083D082F8E4937012740193700DA3A3F2
:101C910093F8740193F5828883E473740293686006
:061CA100EFA3A3A380DF06
:091CA700EBF608EAF608E9F62262
:091CB000EBF0A3EAF0A3E9F02235
:091CB900EBF208EAF208E9F2225C
:00000001FF
